:10000000758150020006C200D294C29612054BD2EE
:10001000961202001201CF12002E12008E12054B12
:100020001200B312054B1200D812054B80EC75126A
:100030002B75130275102875110390029B1200FD99
:1000400075102775162875110075124575130290E5
:1000500002111200FDE510C0E02512F51075120125
:1000600075130290053B1200FDD0E0F510751706E0
:100070007518327519029002F1120149751801754F
:10008000190290053B1201490516D510B9227512C7
:10009000187513037510647511009003551200FD57
:1000A00075121E75130375100075110590042D123D
:1000B00000FD2275121875130375106475110090F8
:1000C000039D1200FD75121E751303751000751146
:1000D000059004871200FD22751218751303751020
:1000E000647511009003E51200FD75121E7513036F
:1000F0007510007511059004E11200FD2285110DA7
:10010000E50D2513F514750C0074211201B2E510EC
:100110001201B2747F1201B274221201B2E50D1203
:1001200001B274071201B2200009E493120195A3F1
:10013000020138E515120195050CE50CB512E8052C
:100140000DE50DB514C0C2002285170DE50D25196A
:10015000F51A750C0074211201B2E5161201B27481
:100160007F1201B274221201B2E50D1201B27407BE
:100170001201B2200009E493120195A3020184E563
:1001800015120195050CE50CB518E8050DE50DB542
:100190001AC0C200227F08D297C29430E705D295D8
:1001A0000201A5C29500D29400000000C29423DF92
:1001B000EA227F08C297C29430E705D2950201C2B5
:1001C000C29500D29400000000C29423DFEA227599
:1001D0000D00750C00742131B2E50C31B2747F3121
:1001E000B2742231B2E50D31B2740731B27400310C
:1001F00095050CE50CB480F5050DE50DB408D3228A
:10020000900554750B19E49331B2A3D50BF831CF97
:1002100022000000E1FDFFFF5E4640E0FEFE7E1E84
:1002200003C1E0707038383838F0F0F0F01800F89A
:10023000F07038303838B8F8780000F0F0703830A6
:100240003838B8F8780020206070F0F8C8800000D6
:10025000C8F87818101008080E0F0F0F00100C0FB8
:100260000F0F0900000F1F1E1C1C1C0C0E1E0F0F71
:100270008BC0787F7F060E0E0E0E070381C0787F3D
:100280007F060E0E0E0E070301383C7C7C7C5C4022
:1002900061733F3F1F07010000000000000004E4FD
:1002A000FCF8F878E0F0F0F070008080C04040404A
:1002B00040C0C080000000C0808080000000C0C03E
:1002C000E020808080804040707F7F7F0761F8FF62
:1002D000BF0701387FFF8783BAFA7A7A13070700CE
:1002E000387E7FFF87C1E07C7F1F1F707C7F3F1FB0
:1002F00000C0E4FCF8180000000484FCFCF4048056
:1003000080C040404040C0C0800000008080C0C02D
:10031000C0C080808080C000C0808080C08040409D
:10032000C0C0804143637B7E7E7E6643030101380B
:100330007FFF8783BAFA7A7A13070778FEF7E3E339
:10034000E16171F17F7F5F076060787F7F474100E7
:10035000060707030300000000040000200000005F
:100360000024000000000040000008000008000019
:10037000080000080000285D3E773E5C0A00000887
:10038000000008000040000008000001000000001C
:100390000092000000000200001000008000000039
:1003A0000200001000008000009200000000000029
:1003B0002000000400000008000008000048001CA5
:1003C0003EB63E1C80090000080000080000001036
:1003D00000000200000000000024000000000004F3
:1003E00000002000000000010000080000400000A4
:1003F000004900000000800000100000020008001A
:10040000000800008800001C3E363E1C000008006A
:1004100000080000080020000004000000000000A8
:1004200000490000000100000800004000800008B2
:10043000008001002000010080080040004000080A
:100440008000010020008100000880880000000872
:1004500040001100000000000000920000000000B9
:10046000000002009000000088E840E200E0680020
:10047000010020002000383C3E3C38000000000015
:1004800010002008002410001000000200004002AC
:10049000004008000020002000000840000100206B
:1004A0000001000010110000001180002200000077
:1004B00000000000490000000000000000082100CA
:1004C000000011E940E408E0680012002820000064
:1004D000383C3E3C3800000010001020011020087D
:1004E00011200000020000800200400008000020EF
:1004F0008000100000048000000040000200202264
:100500000000002200002200000000010000240082
:1005100000000000044002104200000022EA40E017
:1005200008E16800221028200000383C3F3C3800D9
:10053000000020001000221000280200000000002F
:1005400000000000000000000000007DFF7CFFDCD8
:10055000FEDDFA22AED580A83FD300408D142002E4
:0D056000A1C8DA1281CFD9F1DB40A4A6AF0B
:00000001FF
